:100000000C9462000C94D81A0C94051B0C948A0072
:100010000C948A000C948A000C948A000C948A0038
:100020000C948A000C948A000C948A000C948A0028
:100030000C948A000C94A70B0C948A000C948A00F0
:100040000C94321B0C948A000C94AE1E0C94F11E7E
:100050000C948A000C948A000C948A000C948A00F8
:100060000C9408090C948A000000000700020100AB
:100070000003040600000000000000000102040864
:100080001020408001020408102001020408102002
:10009000040404040404040402020202020203032E
:1000A00003030303000000002300260029000000D2
:1000B0000000250028002B0000000000240027007D
:1000C0002A00652011241FBECFEFD8E0DEBFCDBFD0
:1000D00012E0A0E0B1E0EEE3F3E402C005900D927F
:1000E000A63DB107D9F714E0A6EDB2E001C01D921C
:1000F000A03CB107E1F710E0C4ECD0E004C02297C7
:10010000FE010E947A21C23CD107C9F70E94A120BA
:100110000C949D210C9400008091C203813019F44D
:1001200082E08093C2038091C203833019F484E09B
:100130008093C2030895A8950895CF93DF93FC019F
:10014000962F9270862F817060FF20C0992331F026
:100150008091540380831092D60216C0A091D602DB
:10016000C091ED03C770D0E0CE56DD4F8881A8174F
:1001700010F080E03CC081E08A0F8093D602B0E0AE
:10018000AC5FBC4F8C91808381E031C09923C1F07A
:1001900090819093D7021092D602292F207E20368C
:1001A00051F490915403923020F390819F71909379
:1001B000960393E01AC09E3F39F71092540317C07C
:1001C0009091D7029F3F01F79091D602993288F61D
:1001D00021E0290F2093D6023081E92FF0E0EB5384
:1001E000FC4F3083293281F691E090935403DF91E4
:1001F000CF910895DC01ED91FC910190F081E02D0B
:1002000009950895DC01ED91FC910190F081E02DBC
:10021000099508952091C3033091C403382748E01D
:10022000C901880F991F37FF06C09C0151E225279D
:1002300050E1352701C09C01415091F73093C40330
:100240002093C30308958436910520F4BC0180E017
:1002500090E017C09C018E3B910528F42A55310986
:10026000AAE0B0E00CC0823D910528F4245B31097E
:10027000A4E6B0E004C02D5C3109A8E5B2E00E941C
:10028000AE20A4E6B0E09B01AC010E94BD20089521
:1002900090E08C599F4F0E942301089588E080933D
:1002A000EE0380E28093EF031092F00381E08093ED
:1002B000F10382E08093F20383E08093F30382E210
:1002C0008093F40383E28093F5038BE28093F6033B
:1002D00081E28093F70384E28093F80385E28093C0
:1002E000F903089560E08CE00E94401C61E08BE01F
:1002F0000E94401C61E08DE00E94401C60E082E0B2
:100300000E94401C61E084E00E94401C089542E08D
:1003100050E06CE870E080E00E94B81A0895E3E0D5
:10032000F0E089E080935700E491E67081E0E630E8
:1003300009F080E00895CF93DF93C82F0E948F01CA
:10034000882381F0DFB781E08093C103F8940E9495
:100350009B0088E180936000C0936000C1110E94FF
:100360009B00DFBFDF91CF910895FC0140A5842F52
:10037000877090E0959587950196242F217030E045
:10038000820F931F880F880F08958F929F92AF92CC
:10039000BF92CF92DF92EF92FF92CF93FC01C0A564
:1003A000EC2FE770F0E0EE56FD4FA081B0E0C7FF04
:1003B00003C024E130E002C02FE030E0FC0197A14F
:1003C00083E1989FF0011124EA5AFE4F80809180CA
:1003D000A280B380A20FB31F20E43FE14DE750E0BD
:1003E0000E94C820A50194010E9400218C2F8871D1
:1003F00049F469017A01E0EDCE0EE7E0DE1EE11C72
:10040000F11C1BC0C7FF05C060E47AE88CE29EE0E7
:1004100004C060E07EEE8AEB9BE069017A01F8EBB4
:10042000CF0EFBE0DF1EE11CF11CA50194010E9430
:100430000021C20ED31EE41EF51EC701B60169518C
:100440007C4F8F4F9F4F28EE33E040E050E00E94FA
:100450000021A8EEB3E00E94BD20CF91FF90EF9065
:10046000DF90CF90BF90AF909F908F900895DB0169
:10047000FA01582F569590E02481237030E0322FF6
:1004800022274081240F311D11963C932E934481E5
:100490004C70218130E060E4469F200D311D112415
:1004A00013963C932E93129744814073228130E03F
:1004B00060E1469F200D311D112415963C932E932B
:1004C00014974481407C238130E064E0469F200DF6
:1004D000311D112417963C932E9316973596189636
:1004E0009F5F591748F680FF47C040814295469567
:1004F000469543702DE431E0429FC001439F900D2B
:1005000011240C9611969C938E93808190E074E058
:10051000969587957A95E1F783709927829FA00138
:10052000839F500D929F500D1124445F5F4F13968F
:100530005C934E931297808190E09695879596955F
:10054000879583709927829FA001839F500D929F6A
:10055000500D1124445F5F4F15965C934E93149792
:1005600040814370429FC001439F900D11240C961F
:1005700017969C938E9316970895803223E09207E6
:1005800008F1883E23E0920740F48F519340E4E065
:1005900096958795EA95E1F70895803D27E09207C3
:1005A00018F48C5D93400895883928E0920768F428
:1005B000885C974074E0969587957A95E1F78D5021
:1005C0009C4F089580E090E008958FEF93E00895A8
:1005D0008C30910540F4A4E0880F991FAA95E1F7AB
:1005E000885D9C4F0895843F23E0920718F484525D
:1005F0009C4F0895811524E0920740F48657934F4D
:10060000F4E0880F991FFA95E1F7089580E998E0E2
:1006100008959C013695279525753575821B930B9A
:100620009C0123733373969587959695879583736D
:100630009373820F931F9C0154E0369527955A952A
:10064000E1F7280F391F2F703F7041E051E0249FE0
:10065000C001259F900D349F900D1124892F08957E
:100660002D98882319F000002B9A02C000002B98C7
:1006700000002D9A000008952D9A000083B12D9856
:100680000000829581700895CF93DF93D82F5C9AF4
:100690002D985C98C8E08D2F80780E943003DD0F84
:1006A000C150C9F72D98DF91CF9108958F770E949F
:1006B00044030895CF93DF93D82FC8E08D2F80781F
:1006C0000E943003DD0FC150C9F72D98DF91CF9103
:1006D0000895CF93DF932D98C8E080E0D82FDD0FE9
:1006E0000E943C038D0FC150C9F7DF91CF9108954F
:1006F0000E9456030E9469035C9A0895A1E0B0E04D
:10070000E4E8F3E00C945121806869830E9444037B
:100710006981862F0E945A035C9A2196E2E00C942C
:100720006D21CF93C091CE03C827E82FF0E0EB53A3
:10073000FC4F678589E70E947E036C2F8DE30E9442
:100740007E036C2F82E40E947E03CF91089586E29F
:100750000E9478030895CF938BE20E947803C82FFC
:100760008CE20E947803282F30E066E036952795CA
:100770006A95E1F744E0C49FC0011124822B932BBA
:10078000CF910895CF93DF93EC016C818CE10E94AF
:100790007E036D818DE10E947E036E818EE10E9459
:1007A0007E036F8180E20E947E03688581E20E9461
:1007B0007E03698582E20E947E036A8583E20E944D
:1007C0007E036B8584E20E947E036C8585E20E9435
:1007D0007E036D858AE20E947E036E858EE60E940E
:1007E0007E036F858FE60E947E03688980E70E9402
:1007F0007E03698981E70E947E036A8982E70E94FD
:100800007E03DF91CF910895CF92DF92EF92FF9216
:10081000CF93DF936B017C01C11488E3D8068CE988
:10082000E8068CE1F80628F5C701B60120E836E9AC
:1008300048E950E00E940021E901689760E879E604
:1008400087E69FEF0E94D0206C0D7D1D8E1D9F1DA1
:10085000F2E0660F771F881F991FFA95D1F721E7FD
:1008600032E040E050E00E940021F22EE32E80E4CE
:1008700021C0C701B60120E03DE241E351E00E9402
:100880000021E901689760E073ED8EEC9EEF0E9415
:10089000D0206C0D7D1D8E1D9F1D660F771F881F3C
:1008A000991F21E732E040E050E00E940021F22E43
:1008B000E32E80E66C2F6F71680F85E70E947E0340
:1008C0006E2D86E70E947E036F2D87E70E947E03D0
:1008D000DF91CF91FF90EF90DF90CF9008958F92AE
:1008E0009F92AF92BF92CF92DF92EF92FF92CF93FF
:1008F000DF93D82F83E00E9478038093C00384E0C5
:100900000E9478038093BF0360E086E00E947E032C
:1009100061E087E00E947E036FE789E00E947E032A
:1009200065E08AE00E947E0362E18BE00E947E0324
:1009300065E18CE00E947E038091ED0387FF02C099
:1009400067E101C06DEF8DE00E947E0360E08EE004
:100950000E947E03DD2319F083E491E008C020911A
:10096000EC0333E1239FC00111248A5A9E4F0E9459
:10097000C2036CE880E30E947E036FE082E30E9482
:100980007E0362E483E30E947E038091ED0387FF90
:1009900002C064E101C06AE084E30E947E036AE26F
:1009A00085E30E947E036DE286E30E947E0364ED90
:1009B00087E30E947E0360E088E30E947E0360E09C
:1009C00089E30E947E03D11109C0C090CE03D0906C
:1009D000CF03E090D003F090D10307C0C5E9CC2E3F
:1009E000C1ECDC2EED2CCEEDFC2ECAE38F2C99242D
:1009F000AA24BB24682D8C2F0E947E03682D85E0DD
:100A00008C0F0E947E03FE2CED2CDC2CCC24CF5FBF
:100A1000CE3361F76FEF83E40E947E036FEF84E4CF
:100A20000E947E036FEF85E40E947E036FEF86E4F1
:100A30000E947E03DD2311F066E002C06091D203C4
:100A40008DE60E947E0360E089E70E947E0360914C
:100A5000D3038AE70E947E0360E083E70E947E035F
:100A600060E084E70E947E03D11109C06091CA034F
:100A70007091CB038091CC039091CD0304C060ECC6
:100A800072E98DEE99E10E940404DF91CF91FF900D
:100A9000EF90DF90CF90BF90AF909F908F90089590
:100AA00061E087E00E947E0364E28EE70E947E039D
:100AB0008091ED0387FF02C063E801C063E088E036
:100AC0000E947E036091ED03607888E00E947E03BF
:100AD00065E087E00E947E0362E085E00E947E037D
:100AE00083E00E9478038093C00384E00E9478032F
:100AF0008093BF03089583E00E9478038093C0032E
:100B000084E00E9478038093BF0361E087E00E9445
:100B10007E036AE070E080E090E00E94AB1B0E94E0
:100B2000500500000895CF92DF92FF920F931F931C
:100B3000CF93DF931F92CDB7DEB7082F162F8EE32A
:100B400099830E947E03F02EC02E9981D92E8C2D80
:100B50008F19811738F4F60161916F018FE70E94B8
:100B60007E03F5CF64E085E00E947E0383E00E946F
:100B700078038093C00384E00E9478038093BF03CE
:100B80000E94881B6093BB037093BC038093BD03DA
:100B90009093BE0369E087E00E947E0381E080932A
:100BA000C2030F90DF91CF911F910F91FF90DF90C3
:100BB000CF9008950F931F930E9493058091C203D5
:100BC000813099F40E94881B0091BB031091BC03F3
:100BD0002091BD033091BE03601B710B820B930B00
:100BE000603A76488140910548F38091C203813094
:100BF00031F466EB71E086E194E00E944A1D1F919A
:100C00000F9108950F931F938091C203823021F4B6
:100C10001092C20381E020C08091C2038130D9F4D8
:100C20000E94881B0091BB031091BC032091BD035F
:100C30003091BE03601B710B820B930B613A7648B7
:100C40008140910540F061E087E00E947E031092B0
:100C5000C20382E001C080E01F910F910895EF92DE
:100C6000FF920F931F93CF93DF938B019C01442737
:100C700037FD4095542F60E271EA87E090E00E94D2
:100C80002221E9011C161D0614F0C1E0D0E0D801B4
:100C900020E231EA47E050E00E94C8209E0144274C
:100CA00037FD4095542F0E942221790100E010E089
:100CB0000E151F055CF42B9ACE010E94D11B2B98B8
:100CC000CE010E94D11B0F5F1F4FF2CFCDB7DEB711
:100CD000E6E00C946921CF93DF935D9A6091FE0367
:100CE0007091FF0380910004909101040E9404041C
:100CF00060E089E70E947E0361E070E080E090E0C0
:100D00000E94AB1B0E94A703C82F61E070E080E047
:100D100090E00E94AB1B0E94A703D0E0C80FD11D3A
:100D200061E070E080E090E00E94AB1B0E94A703AE
:100D3000C80FD11D61E070E080E090E00E94AB1B25
:100D40000E94A7035D989E01280F311DC901969549
:100D5000879596958795DF91CF910895CF93C82F6A
:100D60005D9A83E00E9478038093C00384E00E9430
:100D700078038093BF0360E086E00E947E0361E019
:100D800087E00E947E036FE789E00E947E0365E0B2
:100D90008AE00E947E0362E18BE00E947E0365E1AF
:100DA0008CE00E947E036DEF8DE00E947E0360E088
:100DB0008EE00E947E036CE280E70E947E0360E08A
:100DC00080E30E947E0360E089E70E947E0365E085
:100DD0008AE70E947E0362E181E70E947E0362E06F
:100DE00082E70E947E0360E083E70E947E0360E06A
:100DF00084E70E947E036091FE037091FF0380915F
:100E00000004909101040E94040467E08DE60E94B2
:100E10007E036AE070E080E090E00E94AB1B69E036
:100E200087E00E947E036AE070E080E090E00E942C
:100E3000AB1BCC2369F0C5E1C15009F459C061E096
:100E400070E088EB91E00E942F060E949B00F4CF97
:100E500061E070E088E891E00E942F060E949B000C
:100E600065E08DE60E947E036AE070E080E090E03D
:100E70000E94AB1B61E070E088EB91E00E942F06BE
:100E80000E949B0064E08DE60E947E036AE070E0B1
:100E900080E090E00E94AB1B61E070E08DE591E0A6
:100EA0000E942F060E949B0062E08DE60E947E0356
:100EB0006AE070E080E090E00E94AB1B61E070E0CF
:100EC0008FEA90E00E942F060E949B0060E08DE672
:100ED0000E947E036AE070E080E090E00E94AB1B1D
:100EE00062E070E085E091E00E942F060E949B0086
:100EF00061E087E00E947E035D98CF910895CF93D3
:100F0000DF93EC014AE050E06D2F70E086E194E061
:100F10000E940F1E6EE286E194E00E942E1DBE012B
:100F200084E0769567958A95E1F76F7077274AE0B8
:100F300050E086E194E00E940F1E6EE286E194E0AC
:100F40000E942E1DBE016F7077274AE050E086E1B7
:100F500094E00E940F1EDF91CF910895D82FC0E03A
:100F6000CD1780F45E9A64E670E080E090E00E9425
:100F7000AB1B5E9864E670E080E090E00E94AB1BE3
:100F8000CF5FEECF6CE271E080E090E00E94AB1B9F
:100F9000E6CF0F931F93CF93DF93EC01062F15E05D
:100FA000115051F0CE010E948721081741F0602FA7
:100FB000CE010E948F21F4CF82E00E94AE07DF9124
:100FC000CF911F910F910895A0E0B0E0EAEEF7E015
:100FD0000C944321482E562EC0E0D0E0612C712C99
:100FE000E12CF12C00E010E0442079F081E048167B
:100FF000A1F092E0491219C028E4622E712C30E26F
:10100000E32EF12C07E513E010C0612C712C6BE18D
:10101000E62EF12C0EEE13E008C04DE1642E712C8B
:1010200059E2E52EF12C05EC13E043018C0E9D1ED8
:101030001092C4031092C3033401A62CA818B12C3B
:10104000C30101966C01AE14BF04A8F4A00EB11E3A
:10105000511006C0C3010E948721F501808305C09D
:10106000F5016081C3010E94C907F50180810E94DA
:101070000A013601E2CFC301511018C0C3010E941A
:101080008721B82EC6010E9487212B2D30E0322FF8
:101090002227282B8091C3039091C40382179307C2
:1010A00079F4C0E0D0E0552453949ECF360160918E
:1010B000C4030E94C9076091C303C6010E94C90707
:1010C000D395C13093E0D90708F48ECF852DCDB7E5
:1010D000DEB7E0E10C945F2160E081E00E94E4076C
:1010E000882331F081E09091C503983309F080E0C6
:1010F000089561E081E00E94E407089561E082E0E4
:101100000E94E407089560E082E00E94E4078111F4
:1011100008C0E7E5F3E01192119283E0E737F807A2
:10112000D1F70895A1E0B0E0E8E9F8E00C9451218E
:1011300089830E944E0192E09093FC039FEF90936D
:10114000FD039AE09093060410920704109208049D
:101150001092FE031092FF031092000410920104FB
:101160002EE1209302049093030428EB3BE030939C
:101170000504209304048981882371F061E080E0F4
:101180000E94E407E7E5F3E01192119283E0E7376C
:10119000F807D1F70E947E082196E2E00C946D21B9
:1011A00060E080E00E94E407811103C081E00E94BA
:1011B00092080895CF93C1E0811101C0C0E06C2F67
:1011C00082E10E94791C6C2F83E10E94791C1092AD
:1011D000B5031092B4038091B9008C6F8093B9006D
:1011E00080E28093B80085E48093BC00CF9108959D
:1011F00085ED8093BC008091BC0084FDFCCF0895F8
:10120000ECEBF0E0108285E480831092B403089543
:101210001F920F920FB60F9211242F933F934F936B
:101220005F936F937F938F939F93AF93BF93EF934E
:10123000FF93CF93DF931F92CDB7DEB78091B900B4
:10124000887F803609F4C7C0A8F5883209F464C0E5
:1012500098F4803109F45DC038F4882309F4F3C0B0
:10126000883009F456C0F1C0883109F455C0803285
:1012700009F0EBC082E0A7C0803409F477C078F4AD
:10128000803309F45FC0883309F0DFC084E08093C5
:10129000B3038091B4038B7F8093B403D0C08035B7
:1012A00009F452C0883509F467C0883409F0CDC00C
:1012B00085E089C0883909F4C0C0A8F4883709F4EA
:1012C0008AC038F4883609F486C0803709F483C0B0
:1012D000BCC0883809F4B1C0803909F47FC08038B7
:1012E00009F0B3C07BC0803B09F493C038F4803A66
:1012F00009F48CC0883A09F48CC0A7C0803C09F47A
:101300009EC0883C09F49BC0883B09F09EC080E0E9
:1013100081C08091B80313C08091B5039FEF980FEF
:101320009093B5038823D1F1E091B603F091B70310
:10133000CF0101969093B7038093B6038081809389
:10134000BB007DC083E03FC0E091B603F091B703DE
:10135000CF0101969093B7038093B6038091BB00B1
:1013600080838091B50381508093B5038091B5034C
:10137000823008F064C061C0E091B603F091B70319
:10138000CF0101969093B7038093B6038091BB0081
:1013900080838091B50381508093B5038091B4031D
:1013A0008B7F8093B4038091B40380FF4CC0809105
:1013B000B4038E7F8093B4038091B40382608093E2
:1013C000B40384EA3DC08093B3038091B4038B7F60
:1013D0008093B40338C01092B50331C0E091B903D3
:1013E000F091BA03309749F18091BB0089838091D5
:1013F000B50391E0980F9093B503811102C062E0AC
:1014000001C060E0CE010196099515C00E94F80860
:1014100016C081E0E091B903F091BA03309769F00A
:10142000882311F063E001C061E0CE0101960995C7
:1014300099819093BB00811102C085E801C085ECC1
:101440008093BC0002C00E94F8080F90DF91CF91FA
:10145000FF91EF91BF91AF919F918F917F916F918C
:101460005F914F913F912F910F900FBE0F901F9062
:1014700018958F929F92AF92BF92CF92DF92EF9288
:10148000FF92CF93DF93EC010E94881B6B017C01DC
:101490004E01A12CB12C8091B40382FF11C0209782
:1014A000D1F30E94881B6C197D098E099F0986164D
:1014B0009706A806B90678F70E94000981E004C0E3
:1014C0008091B3031092B303DF91CF91FF90EF901F
:1014D000DF90CF90BF90AF909F908F900895A2E043
:1014E000B0E0E5E7FAE00C944D21182F7B01022FC4
:1014F000047022FD05C080910B0190910C0102C087
:1015000080E090E02A8349830E94390A2A81498138
:10151000811136C01092B3034093B503F092B70324
:10152000E092B603110F1093B8039091B40321FF1A
:1015300002C085E001C084E0892B8093B4038091D0
:10154000B40381FF0BC08091B4038D7F8093B403FB
:101550008091B8038093BB0085EC01C085EE809339
:10156000BC00822F817020FF0BC0011105C080914B
:101570000B0190910C0102C080E090E00E94390ABA
:101580002296E6E00C946921A2E0B0E0EAECFAE0F1
:101590000C944D21182F7B01022F047022FD05C0F1
:1015A00080910B0190910C0102C080E090E02A83B1
:1015B00049830E94390A2A814981811138C01092D9
:1015C000B3034093B503F092B703E092B603812FC3
:1015D000880F81608093B8039091B40321FF02C00B
:1015E00085E001C084E0892B8093B4038091B4032B
:1015F00081FF0BC08091B4038D7F8093B4038091F1
:10160000B8038093BB0085EC01C085EE8093BC00DD
:10161000822F817020FF0BC0011105C080910B014A
:1016200090910C0102C080E090E00E94390A22965D
:10163000E6E00C946921A0E0B0E0E1E2FBE00C946C
:101640004B210E94881B0091AF031091B0032091A1
:10165000B1033091B2036B017C01C01AD10AE20AD6
:10166000F30A9701860141E1C41647E2D406E1047A
:10167000F10408F442C02091AE0331E0320F309300
:10168000AE0320FF02C017E001C010E06093AF037B
:101690007093B0038093B1039093B20363E070E062
:1016A00086E194E00E94020161E070E086E194E04E
:1016B0000E94020107E0010F812F90E0EC01CC0FA6
:1016C000DD1FC35FDE4F68817981672F77276370E5
:1016D0007727880F991F880F991F682B792B86E130
:1016E00094E00E94FA0068817981772786E194E08E
:1016F0000E94FA001F5F1013DFCFCDB7DEB7E8E01E
:101700000C94672125B190E0FC01EE0FFF1FE80F5C
:10171000F91FE25EFC4F8081282B25B988B19181A9
:10172000892B88B98BB19281892B8BB9089585B1AA
:1017300090911B03892385B988B190911C0389235B
:1017400088B98BB190911D0389238BB908951F929D
:101750000F920FB60F9211242F933F934F935F93E5
:101760006F937F938F939F93AF93BF93CF93EF9399
:10177000FF93C0917A0380910601C81708F03EC01C
:101780008091190390911A039093870080938600AB
:10179000EC2FF0E0EE0FFF1FE35FFE4F80819181A1
:1017A0000E94E802880F991F90931A0380931903EF
:1017B0008091190390911A0320910701309108013B
:1017C000281B390B309308012093070180910404F2
:1017D00090910504880F991F2817390720F49093DA
:1017E00008018093070180917803811142C08091A4
:1017F000FC0380FF41C0C830E0F53EC08091190372
:1018000090911A039093870080938600809107013E
:101810009091080190931A038093190380917803A3
:10182000882319F08FEF9FEF06C0809119039091E4
:101830001A0388559240909389008093880080E431
:101840009CE9909308018093070180918400909116
:1018500085008097D0F30E94970B809179038111C6
:1018600005C08091060181500E94820B10927A037C
:1018700027C08FEF9FEF06C08091190390911A0344
:1018800088559240909389008093880080918400CD
:10189000909185008097D0F30E94970B80917903F7
:1018A000811104C080917A03811106C080917A036E
:1018B0008F5F80937A0304C081500E94820BF6CF21
:1018C000FF91EF91CF91BF91AF919F918F917F91B8
:1018D0006F915F914F913F912F910F900FBE0F909D
:1018E0001F90189524E0829FC00111248C3091052F
:1018F00038F0853F23E0920728F084EF93E00895C5
:101900008CE090E00895CF93DF93C091FD03C03346
:1019100090F48C2F807339F0803141F480917B03F7
:101920008295807F05C08091800302C080918103F1
:10193000CF70D0E015C0CF33E0F4CF70D0E080910D
:101940007B038295807F0E94720CDE01AA0FBB1F71
:10195000A35FBE4F11969C938E9321968091810335
:101960000E94720CFE01EE0FFF1FE35FFE4F91839A
:101970008083DF91CF91089580917C0390917D03C6
:101980009F770E94090380937B038F3029F4809115
:1019900081038695805804C099E0899F802D112489
:1019A00080938003F8940E94830C78948091F703CD
:1019B0008132E1F4809180039FEF980F9E3F78F091
:1019C0008091B0008F7D8093B00061E080918003B2
:1019D000811101C060E083E00E94791C089580932A
:1019E000B4008091B00080628093B0000895FF92AF
:1019F0000F931F93CF93DF930FEE13E0C0E0D0E07F
:101A0000B3E0FB2E8C2FD801ED918D019E2F907F9E
:101A10009031F1F4EF70F0E0EE0FFF1FE35FFE4F47
:101A2000208131816F2D0E94E020E92FF0E0EE0F40
:101A3000FF1FE457FD4F61E080819181821793077A
:101A400008F060E0FE01E656FD4F80810E94791C9F
:101A50002196CB30D105B1F6CDB7DEB7E5E00C94D9
:101A60006A210F931F93CF93DF9307E513E0C0E044
:101A7000D0E02091FD03822F8F7090E0C817D90726
:101A8000E9F00196C817D90711F42033B8F4F8012A
:101A9000808191819F70892B79F0F894F801808181
:101AA00091819F700E94BD02FE01EE0FFF1FE35F58
:101AB000FE4F9183808378940E94F70C21960E5FED
:101AC0001F4FC031D105A9F6DF91CF911F910F9122
:101AD0000895FF920F931F93CF93DF9385EC93E0CC
:101AE0000E94B501809306019091FD03292F2F706C
:101AF000281304C081E0820F8093060190539F3029
:101B000060F44091060130E0842F90E0019728179F
:101B1000390719F44F5F4093060180910601813126
:101B200018F080E180930601E0E2F3E0DF01129714
:101B30001C92DF0111971C921082339683E0E134EE
:101B4000F807A1F74FEF3FEFA7EAB2E00FEE13E07F
:101B50002FEFE80189918E018031F8F490E0FD01CA
:101B600032976081FC01EE0FFF1FE80FF91FE25E64
:101B7000FC4F8081862B8083CD010197EC01588139
:101B80008181852B81839C918281892B82836095C1
:101B9000509590952923352346231396D3E00A3F89
:101BA0001D07B9F640931B0330931C0320931D03BC
:101BB000CAE9D2E00FEE13E0F12CF80181918F0118
:101BC000823230F08632B8F0863211F460E010C014
:101BD000F9E0FF1204C08091C1008F7E06C08AE048
:101BE000F81205C08091C100877F8093C10061E039
:101BF00088810E94401CF3942196EBE0FE12DDCF19
:101C00008091EF03803231F461E089E00E94791C19
:101C100082E801C082E08093800081E080937903B4
:101C2000809378038091F703813211F08732D9F4E1
:101C300061E083E00E94401C60E083E00E94791C28
:101C40008091F703813231F481E08093B00080937A
:101C5000B10009C082E08093B00085E08093B100BC
:101C60008EE38093B3008AE1809381008FEF9FEF32
:101C7000909389008093880080ED97E0909387008F
:101C80008093860080E49CE990930801809307018B
:101C900090931A038093190310927A0380916F0036
:101CA000816080936F008091FC0383FF0DC0809161
:101CB0005703909158039F70892B31F00E94310D8A
:101CC0001092780310927903CDB7DEB7E5E00C945B
:101CD0006A21CF93C82F8091F6038B3221F46C2FA9
:101CE0008AE00E94791C8091F703873249F4809141
:101CF000B000CC2311F0806101C08F7E8093B000D2
:101D0000CF910895A2E2B0E0E8E8FEE00C94412112
:101D10006B017C010E947C1B4B015C0181E00E94F5
:101D20006F0483E08093C2030E947B0562EC71E044
:101D300086E194E00E944A1D7BE1272EE0E53E2EDD
:101D4000F7E47F2EA6E44A2EB5E55B2EC114D1043C
:101D5000E104F10469F00E947C1B681979098A0981
:101D60009B096C157D058E059F0510F080E0D4C0A1
:101D70008091C203843051F760ED71E086E194E018
:101D80000E944A1D8FE70E9456030E9469038AA39E
:101D9000823601F505EC13E00E946903D8018D93AA
:101DA0008D01B3E00E3E1B07B9F78091C503883360
:101DB00009F0ACC069ED71E086E194E00E944A1D33
:101DC00082E48AA361E0CE0182960E94DA055D9AE0
:101DD00081E0A2C0803741F0893611F581E00E9490
:101DE000920889E4898304C03982C12CD12C760100
:101DF0009091C1038091FC03992311F0806801C088
:101E00008F778093FC03EEEEF3E0DE011296822DD5
:101E100001900D928A95E1F76CE1CE01019674C0B4
:101E20008437D9F4E4E5E98383E08A8388E88B8307
:101E30008BE08C838D8386E1EDE2F1E0DE01169686
:101E400001900D928A95E1F76BE1CE0101960E9417
:101E5000DA05C12CD12C760159C0853789F40EEEF4
:101E600013E00E946903D8018D938D01B4E009301D
:101E70001B07B9F761E080E00E94E4075AA241C065
:101E80008636B9F44982E7E5F3E0AE014D5F5F4F76
:101E9000208131813296CA010197DC013C93DA013D
:101EA0002C934E5F5F4FB3E0E737FB0789F761E2A2
:101EB000B4CF8736C9F407E513E00E946903682EA2
:101EC0000E946903262D30E0322F2227280F311D72
:101ED000F801219331938F01F3E007371F0769F76A
:101EE0007AA20E947E080DC0873481F4E7E5F3E012
:101EF0001192119283E0E737F807D1F70E947E082C
:101F00007AA261E0CE0182960E94DA0583E0809396
:101F1000C2030E9450051ACFA296E2E10C945D2103
:101F20001F93CF93DF93C82FD62F61E00E94401CF0
:101F300061E08C2F0E94791C61E08D2F0E94791C3A
:101F40008AE090E00E94D11B8D2F0E94AC1C892B4F
:101F500071F060E08C2F0E94791C8AE090E00E9472
:101F6000D11B8D2F0E94AC1C11E0892B09F010E0D1
:101F700060E08C2F0E94401C60E08C2F0E94791C36
:101F800060E08D2F0E94791C812FDF91CF911F91EE
:101F9000089580E48093BA001092BD008DE990E02E
:101FA0009093BA038093B9031092540315E004E0B0
:101FB000C2E0FC2E80915403813039F480E00E940D
:101FC0006F04F09254035E98F5CFC0915403C33070
:101FD00061F45D98809196030E949103C093C203BF
:101FE0000E94500500935403E5CF80915403843040
:101FF00009F78091C2038430E9F68FE70E94560307
:10200000C4E0D3E0E091ED03E770F0E0EE56FD4F61
:10201000808190E09E01245033402817390724F432
:102020000E9469038993EECF109354035D9AC2CF47
:10203000AAE2B0E0EEE1F0E10C9450211FEF198329
:1020400089E2E5ECF3E0DE01129601900D928A95AB
:10205000E1F721E04AE2BE016F5F7F4F80E20E941C
:102060006F0A81110EC021E041E0BE016F5F7F4F1A
:1020700080E20E94C40A811104C082E0809354036C
:1020800002C01093540380915403823051F00E9497
:102090007C1B609350037093510380935203909381
:1020A0005303AA96E3E00C946C21A1E0B0E0EBE5C9
:1020B000F0E10C945121809154038230D9F4809145
:1020C0009603805A898321E041E0BE016F5F7F4F14
:1020D00080E20E946F0A882369F08FEF8093540397
:1020E0000E947C1B609350037093510380935203B2
:1020F000909353032196E2E00C946D21A1E0B0E0AF
:10210000E4E8F0E10C945121809154038230D1F441
:1021100021E041E0BE016F5F7F4F80E20E94C40A70
:10212000882371F08FEF809354030E947C1B60938F
:10213000500370935103809352039093530302C052
:10214000898101C08FEF2196E2E00C946D21A2E21B
:10215000B0E0EDEAF0E10C9441219E012F5F3F4F8A
:1021600080E1D9011D928A95E9F764EE71E086E17C
:1021700094E029A33AA30E944A1D0E947B051D8A70
:102180001E8A1F8A188E312C212C00E0812C912C64
:10219000540180E4482E81EE582E8DE9682E88E1A6
:1021A000782E90E5C92E93ECD92EE12CF12C84EFFA
:1021B00091E0A0E0B0E08D8F9E8FAF8FB8A380EC50
:1021C00091EDA8E9BBE1898F9A8FAB8FBC8F80E43A
:1021D00091EEADE9B8E1898B9A8BAB8BBC8B86E134
:1021E00094E00E94161E892B09F4E1C086E194E078
:1021F0000E94431E9C0133272C32310509F442C052
:10220000ACF42332310509F0ABC019821A821B826B
:102210001C821D821E821F82188619861A861B86C2
:102220001C861D861E861F86188A60C024343105D0
:1022300029F02335310509F4B2C092C064E486E187
:1022400094E00E942E1D2AE030E040E451EE6DE95A
:1022500078E186E194E00E94AA1D6CE286E194E0B8
:102260000E942E1D2AE030E040EC51ED68E97BE150
:1022700086E194E00E94AA1D6CE286E194E00E944F
:102280005C1DADCF0F5F043009F0A9CF29813A81E1
:102290004B815C81A8EEB3E00E94BD20698B7A8BF4
:1022A0008B8B9C8B2D813E814F8158850E94BD2058
:1022B000698F7A8F8B8F9C8F29853A854B855C85BA
:1022C0002D8F3E8F4F8F58A32D853E854F85588982
:1022D0000E94BD206B017C0160323EE473078105E2
:1022E000910530F462E38CE10E947E0300E077CF39
:1022F000603345E774078105910510F462E2F3CF7E
:1023000060345CE975078105910510F466E2EBCF56
:1023100080E5C81683ECD806E104F10410F462E10C
:10232000E2CF90E6C9169AEED906E104F10410F462
:1023300065E1D9CFA0E7CA16A1E1DA06A1E0EA0675
:10234000F10410F461E0CFCFB0EACB16B6E8DB06BB
:10235000B1E0EB06F10410F463E0C5CF65E0C3CF54
:1023600010ED180F1A3008F03ACFE1E0F0E0EC0F72
:10237000FD1F24E0029FE00DF11D11242081318119
:1023800042815381AAE0B0E00E94BD20610F711D1F
:10239000811D911D608371838283938320CF49883F
:1023A0005A886B887C88812C912C540118CF811419
:1023B0009104A104B10489F4C301B2010E94040490
:1023C00061E070E080E090E00E94AB1B1D8A1E8AF5
:1023D0001F8A188E312C22242A948D8D9E8DAF8DCC
:1023E000B8A188169906AA06BB06D0F40E94A703D6
:1023F0002D893E894F89588D280F311D411D511D52
:102400002D8B3E8B4F8B588F381608F4382E821543
:1024100008F4282E3FEF831A930AA30AB30A56C082
:10242000C301B20128EE33E040E050E00E940021F9
:10243000BA01A9012AE030E086E194E00E94F81D8B
:102440006CE286E194E00E942E1D4AE050E0632D8C
:1024500086E194E00E94071E6CE286E194E00E940F
:102460002E1D6D897E898F89988DA50194010E940A
:102470000021BA01A9012AE030E086E194E00E943F
:10248000F81D6CE286E194E00E942E1D4AE050E0C7
:10249000622D86E194E00E94071E6CE286E194E0E2
:1024A0000E945C1D4C0C5D1C6E1C7F1C898D9A8DDE
:1024B000AB8DBC8D84159505A605B70520F449881C
:1024C0005A886B887C88812C912C540129893A89FF
:1024D0004B895C89283E33404105510509F07FCE88
:1024E000A296E2E10C945D21A1E0B0E0EAE7F2E11E
:1024F0000C94512180E00E949B0161E085E00E94E4
:10250000401C61E086E00E94401C0E94720160E075
:1025100080E00E94401C61E081E00E94401C40E09D
:1025200052EC61E070E086E194E00E945E1F0E9440
:10253000D0080E94830861EF71E086E194E00E9478
:102540002B1D88E893E00E947F0768E072E086E137
:1025500094E00E942B1D4AE050E069E070E086E1C3
:1025600094E00E94E01D0E94870178945E9A60E1E9
:102570008FE00E94900F882329F05E985D980E945A
:10258000A710FBCF6EE089E00E94900F811104C07C
:102590000E946C08811119C06BE472E086E194E03E
:1025A0000E942B1D60E070E0CB010E94820E882308
:1025B00049F00E94790860E172E086E194E00E94AF
:1025C0004A1D5D9A0E94690D10C00E94690D80919C
:1025D000F403823209F0C6C08091F503833209F01A
:1025E000C1C08091FC0381FDC3C08091F40382329D
:1025F00031F58091F503833211F581E00E94DA080C
:102600008091FC0382FF08C06BE272E086E194E0F7
:102610000E944A1D0E94C90F64E170E080E090E0D2
:102620000E94AB1B21E041E0BE016F5F7F4F80E263
:102630000E94C40A811103C081E08093540366E3C1
:1026400072E086E194E00E942B1D8FE00E949B01C6
:1026500080E00E946F041092960380E00E94910334
:1026600080E0883170F08093D80283E08093C203C9
:102670000E947B0580915403882371F00E941810FA
:102680000BC021E0280FE82FF0E0EB53FC4F9785BB
:10269000992349F3822FE5CF8091F903982F9D7FED
:1026A000983229F440E052EC61E070E023C08932B6
:1026B00051F42EE240EA56E861E070E086E194E0F1
:1026C0000E94DF1F1BC08091ED038871803129F4C7
:1026D00040E855E260E070E00DC04091C6035091C3
:1026E000C7036091C8037091C9034A305105610561
:1026F000710570F386E194E00E945E1F86E194E02C
:102700000E94161E892B29F086E194E00E94431E48
:10271000F5CF8091F803843229F08091C1008F7E3B
:102720008093C1008091F903853241F08852833053
:1027300028F08091C100877F8093C1001092DA0257
:102740001092D902109256030E94881B6093920344
:102750007093930380939403909395032196E2E002
:102760000C946D218091FC038B7F8093FC0339CF07
:1027700082FD3BCF64EF71E080E090E00E94820E2A
:10278000882309F432CF0E94790860E172E086E183
:1027900094E00E944A1D0E94690D5D9A26CFCF9356
:1027A000DF9386E194E00E94161E892BE9F0C09128
:1027B000D902D0E0CE0101968F7199272091DA02DB
:1027C00030E08217930781F086E194E00E94431E77
:1027D000C552DD4F88838091D90290E001968F71B8
:1027E00099278093D902DDCFDF91CF910895A0E0A2
:1027F000B0E0EDEFF3E10C944B21D82FC62F0E94EF
:10280000881B0091AF031091B0032091B103309168
:10281000B2036B017C01C01AD10AE20AF30A9701E4
:10282000860141E1C41647E2D406E104F10408F44C
:10283000D1C16093AF037093B0038093B1039093C1
:10284000B20380910D0190910E01880F991F809322
:102850009703892F877020919803287F282B209336
:10286000980380910F0190911001880F991F382FC4
:10287000330F330F330F2770232B20939803282F08
:1028800022952695277080919903807C9770990FE7
:10289000990F990F822B892B809399032091110115
:1028A00030911201220F331F922F9295990F990F99
:1028B000907C8F73892B80939903932F9295990F16
:1028C000990F907C822F86958695892B80939A0309
:1028D00032FB882780F920919B032E7F282B2093A1
:1028E0009B038091130190911401880F991F382F39
:1028F000330F2170232B20939B03382F331F332753
:10290000331F20919C03207F892F8770880F232BF2
:10291000282B20939C038091150190911601880F1C
:10292000991F382F3295307F2F70232B20939C03D3
:10293000382F32953F7020919D032078892F877022
:102940008295807F232B282B20939D038091170154
:1029500090911801880F991F2F7720939D03292F9D
:102960002795222727958695822B80939E03892F72
:102970008695837020919F032C7F282B20939F03A3
:102980008091190190911A01880F991F382F330FE8
:10299000330F2370232B20939F03382F32953695C6
:1029A000369533702091A003207E892F8770880F81
:1029B000880F232B282B2093A00380911B0190913B
:1029C0001C01880F991F382F3295330F307E2F71DD
:1029D000232B2093A0039295990F907E8695869540
:1029E0008695892B8093A10380911D0190911E01F2
:1029F000880F991F8093A203892F87702091A303CA
:102A0000287F282B2093A30380911F019091200100
:102A1000880F991F382F330F330F330F2770232B55
:102A20002093A303282F2295269527708091A40335
:102A3000807C9770990F990F990F822B892B809327
:102A4000A4032091210130912201220F331F922FE4
:102A50009295990F990F907C8F73892B8093A40383
:102A6000932F9295990F990F907C822F869586953A
:102A7000892B8093A50332FB882780F92091A60338
:102A80002E7F282B2093A60380912301909124016F
:102A9000880F991F382F330F2170232B2093A60303
:102AA000382F331F3327331F2091A703207F892F0F
:102AB0008770880F232B282B2093A7038091250153
:102AC00090912601880F991F382F3295307F2F70F3
:102AD000232B2093A703382F32953F702091A80312
:102AE0002078892F87708295807F232B282B209335
:102AF000A8038091270190912801880F991F2F77B3
:102B00002093A803292F2795222727958695822B86
:102B10008093A903969593708091AA038C7F892B4B
:102B20008093AA032091290130912A01220F331F9B
:102B3000922F990F990F8370892B8093AA03229566
:102B40002695269523708091AB03807E932F9770F6
:102B5000990F990F822B892B8093AB0320912B0126
:102B600030912C01220F331F922F9295990F907E56
:102B70008F71892B8093AB03832F8295880F807E82
:102B8000269526952695282B2093AC03DD2311F05E
:102B900088E001C080E0CC2311F094E001C090E017
:102BA000892B8093AD036FE070E086E194E00E9492
:102BB0000201C7E9D3E0699186E194E00E94701EAA
:102BC00083E0CE3AD807B9F760E070E086E194E0A0
:102BD0000E940201CDB7DEB7E8E00C946721CF93E5
:102BE000C82F682F86E194E00E94701E8C2F0E94EF
:102BF0000A01CF910895A0E0B0E0E1E0F6E10C9485
:102C00004B21C82F0E94881B0091AF031091B00385
:102C10002091B1033091B2036B017C01C01AD10A3B
:102C2000E20AF30A9701860141E1C41647E2D4069D
:102C3000E104F10408F445C06093AF037093B0035E
:102C40008093B1039093B2031092C4031092C30314
:102C500088EA0E94EF15CC2311F081E801C081E0E1
:102C60000E94EF1580E10E94EF1500E010E0F801EE
:102C7000EE0FFF1FE35FFE4F808191810E94E8020B
:102C8000EC01B3E0CC0FDD1FBA95E1F78D2F0E9468
:102C9000EF158C2F0E94EF150F5F1F4F00311105AC
:102CA00031F76091C40370E086E194E00E94FA007D
:102CB0006091C3037091C403772786E194E00E947A
:102CC000FA00CDB7DEB7E8E00C946721AAE1B0E0E6
:102CD000ECE6F6E10C9443210E949B008CE00E94FC
:102CE000780381110BC064E872E086E194E00E94F1
:102CF0004A1D80E00E946F040E947B050E94CF1352
:102D00000E94881B0E947E1091E0853009F090E0BF
:102D10001FEF8091C203843009F406C2911104C2EE
:102D200084C00E94AB0390937F0380937E035D9ADF
:102D3000C0929203D0929303E0929403F092950391
:102D40001092550310928603109287031092880305
:102D50001092890380917C0390917D03880F991FC5
:102D6000816090937D0380937C035E9880E00E9455
:102D7000690E80910403982F9E7309F02CC2F89479
:102D80008091ED0345E053E06DE071E087700E94B3
:102D900037020E94830C78949091040380914E0333
:102DA00090FF13C2811124C097E5E92E93E0F92E1C
:102DB00000E010E0F7018081918194FD0CC0F801E2
:102DC000EE0FFF1FE35FFE4F808191810E94E802BA
:102DD000D7018D939C930F5F1F4FB2E0EB0EF11C58
:102DE0000031110539F70E947E0881E080934E037F
:102DF00080915603811103C081E0809356031092A5
:102E0000770310927903109278038091ED03887113
:102E100009F009C20E94F70C83E08093C2030E946C
:102E2000500581E080934F035D980E94881B4B0101
:102E30005C010E947C1B6B017C01809155038230F8
:102E400008F063C040909203509093036090940305
:102E50007090950380918E0390918F03A0919003C1
:102E6000B091910384159505A605B70509F44DC0E9
:102E700085EC93E00E94C5016C5D75408109910964
:102E8000950184010419150926093709601771078E
:102E900082079307D0F540928E0350928F03609281
:102EA0009003709291030E94A703282F80938203BE
:102EB0008091830390918403820F911D90938403EA
:102EC00080938303609185036F5F6093850369300E
:102ED000E0F070E00E94EC20709384036093830321
:102EE00080918103E3E08E9F600D711D1124769522
:102EF000679576956795609381030E94BC0C10924C
:102F000084031092830310928503809156030091ED
:102F1000D802882351F110915503101708F029C2E7
:102F200040909203509093036090940370909503A7
:102F3000A501940124193509460957092F8B388FAB
:102F4000498F5A8F85EC93E00E94C50168517C4FF0
:102F50008F4F9F4F2F89388D498D5A8D6217730778
:102F60008407950708F4CCC104C280919203909124
:102F70009303A0919403B091950375016401C81A5D
:102F8000D90AEA0AFB0A85EC93E00E94C5019B017D
:102F9000AC01A02FB0E00E94BD206C157D058E0510
:102FA0009F0558F48092920390929303A092940309
:102FB000B092950381E080934F0380917803811153
:102FC00016C08091F903883219F40E941B0B0FC0C0
:102FD000893239F460915503809177030E94F71389
:102FE00006C08A3221F4809177030E94FB158091FC
:102FF0004F03882309F472C0E0919603EF5FE093DA
:103000009603E83131F0F0E0EB53FC4F87858111F6
:1030100002C0109296038091FE039091FF03A0914D
:103020000004B0910104892B8A2B8B2B09F44EC02C
:103030008091860390918703A0918803B0918903C2
:10304000892B8A2B8B2B09F441C00E946B06082F19
:1030500010E02091090130910A01369527953695A7
:1030600027952C5E3F4F2017310770F40E947C1B80
:1030700068517C4F8F4F9F4F6093860370938703F7
:103080008093880390938903C801880F991F880F44
:10309000991F4091090150910A019A01220F331F93
:1030A000240F351F820F931F9695879596958795C8
:1030B00090930A01809309016091CA037091CB0338
:1030C0008091CC039091CD030E94040480919603DB
:1030D0000E9491030E94551010924F038091540357
:1030E0008F3F09F041C20E947C1B00915003109158
:1030F00051032091520330915303601B710B820BDB
:10310000930B693E73408105910508F42DC20E941E
:103110007C1B6093500370935103809352039093F0
:1031200053030E94181020C20E94881B6B017C016F
:103130008091C2038430D1F48FE70E94560304E0EB
:1031400013E0E091ED03E770F0E0EE56FD4F808173
:1031500090E0980124503340281739070CF0E1CD56
:103160000E946903D8018D938D01EBCFE091ED03AF
:10317000E770F0E0EE56FD4F40814F5F21E0BE0169
:103180006F5F7F4F80E20E94C40A882371F0109322
:1031900054030E947C1B60935003709351038093EF
:1031A00052039093530390E0B4CDE091ED03E770A8
:1031B000F0E0EE56FD4F408150E0BE016E5F7F4F64
:1031C00084E093E00E947E21B3CD882309F410CEE1
:1031D00010924E030DCE982F9873983309F008CEB5
:1031E0009091FB02892787FF03CE90589093FB02B2
:1031F0008091F903853209F0FBCD10E0212F30E0FA
:1032000080910403877090E0821793070CF4F0CD4F
:103210001F5FE12FF0E0EC5FFC4F608186E194E0FE
:103220000E94701EEBCF8091FB02909104039827BF
:1032300096FD5AC0807C90E489278093FB028091A0
:10324000DA023091D9028317D1F0ECEFF2E020E0FE
:103250002F5F90E0DC01A552BD4F4C914193019648
:103260008F719927283011F08313F2CF8093DA02FF
:10327000295C8091FB02282B2093FB0235C08091B2
:1032800082038093FC028091F403863251F482E140
:103290000E94D51C95958795959587958093FD02FD
:1032A00002C01092FD028091F503863251F483E151
:1032B0000E94D51C95958795959587958093FE02DC
:1032C00002C01092FE0280917E0390917F03909342
:1032D000FF028093000380917C0390917D039F7790
:1032E0000E9409038093010369E08BEF92E00E9442
:1032F00093050E94020681118DCD0E94CF13F9CF54
:1033000080917C0390917D03880F991F90937D039A
:1033100080937C0381E080934F03111110C0C09211
:103320008A03D0928B03E0928C03F0928D0310926B
:1033300086031092870310928803109289031F5FFF
:103340001093550385EC93E00E94C501640D751D33
:10335000861D971D6093920370939303809394034B
:10336000909395035E9A81E00E94690E0E94BC0CC6
:1033700003C0101709F4A7C080915503882309F4EE
:103380001CCE809106048823D9F090917703911187
:1033900017C040918A0350918B0360918C03709108
:1033A0008D0346015701841A950AA60AB70A90E0D0
:1033B0000E942301681579058A059B0508F4B5C0AC
:1033C000809108048823D9F090917903911117C056
:1033D00040918A0350918B0360918C0370918D030F
:1033E00046015701841A950AA60AB70A90E00E947E
:1033F0002301681579058A059B0508F4ADC0809105
:1034000007048823D9F090917803911117C0409157
:103410008A0350918B0360918C0370918D03460158
:103420005701841A950AA60AB70A90E00E94230160
:10343000681579058A059B0508F492C08091FE0302
:103440009091FF03A0910004B0910104892B8A2B75
:103450008B2B09F4B2CD8091860390918703A091C4
:103460008803B09189030097A105B10509F4A5CDA2
:10347000C81AD90AEA0AFB0AF7FC9FCD8091FC031F
:10348000829581700E94AE0680E00E946F040E94C7
:1034900050050E947C1B6B017C012091030430E0ED
:1034A000A8EEB3E00E94AE20C60ED71EE81EF91E9D
:1034B0006894C0F8C0928603D0928703E092880394
:1034C000F09289037ACD8091920390919303A09119
:1034D0009403B091950324013501481A590A6A0AE8
:1034E0007B0A85EC93E00E94C5019B01AC01A12FF2
:1034F000B0E00E94BD20641575058605970508F0AB
:103500003BCF10927D0310927C0381E080934F03A8
:10351000109281030E94BC0C8092920390929303BC
:10352000A0929403B092950327CF81E08093770314
:103530000E94310D809102040E9448016C0D7D1D96
:103540008E1D9F1D61606093860370938703809337
:1035500088039093890334CF81E0809379034FCF20
:1035600081E0809378036ACF6A96E0E10C945F2152
:103570008230E8F4E82FF0E0EE0FFF1FE75FFB4F2B
:1035800071836083813041F0809169008C7F842B4E
:1035900080936900E89A089580916900440F551F4F
:1035A000440F551F837F842B80936900E99A089507
:1035B0001F920F920FB60F9211242F933F934F93A8
:1035C0005F936F937F938F939F93AF93BF93EF938B
:1035D000FF938091090490910A04892B29F0E091CE
:1035E0000904F0910A040995FF91EF91BF91AF9101
:1035F0009F918F917F916F915F914F913F912F910B
:103600000F900FBE0F901F9018951F920F920FB63C
:103610000F9211242F933F934F935F936F937F9358
:103620008F939F93AF93BF93EF93FF9380910B047E
:1036300090910C04892B29F0E0910B04F0910C047B
:103640000995FF91EF91BF91AF919F918F917F91DC
:103650006F915F914F913F912F910F900FBE0F90FF
:103660001F9018951F920F920FB60F9211242F934F
:103670003F938F939F93AF93BF9380910E0490914C
:103680000F04A0911004B091110430910D0423E0B7
:10369000230F2D3720F40196A11DB11D05C026E88A
:1036A000230F0296A11DB11D20930D0480930E04DB
:1036B00090930F04A0931004B0931104809112040E
:1036C00090911304A0911404B09115040196A11DCA
:1036D000B11D8093120490931304A0931404B0932B
:1036E0001504BF91AF919F918F913F912F910F90B2
:1036F0000FBE0F901F9018952FB7F89460910E048D
:1037000070910F0480911004909111042FBF0895BF
:103710003FB7F8948091120490911304A09114047F
:10372000B091150426B5A89B05C02F3F19F001964E
:10373000A11DB11D3FBF6627782F892F9A2F620FD9
:10374000711D811D911D42E0660F771F881F991F13
:103750004A95D1F70895CF92DF92EF92FF92CF93DF
:10376000DF936B017C010E94881BEB01C114D10423
:10377000E104F10479F00E94881B6C1B7D0B683E0C
:103780007340A0F381E0C81AD108E108F108C851DC
:10379000DC4FECCFDF91CF91FF90EF90DF90CF9097
:1037A00008950197009739F0880F991F880F991F86
:1037B00002970197F1F70895789484B5826084BDEB
:1037C00084B5816084BD85B5826085BD85B5816025
:1037D00085BDEEE6F0E0808181608083E1E8F0E085
:1037E0001082808182608083808181608083E0E8B4
:1037F000F0E0808181608083E1EBF0E08081846093
:103800008083E0EBF0E0808181608083EAE7F0E094
:1038100080818460808380818260808380818160F8
:1038200080838081806880831092C10008958330F6
:1038300081F028F4813099F08230A1F0089586302B
:10384000A9F08730B9F08430D1F4809180008F7D69
:1038500003C0809180008F7780938000089584B5A5
:103860008F7702C084B58F7D84BD08958091B000AC
:103870008F7703C08091B0008F7D8093B000089552
:10388000CF93DF9390E0FC01E458FF4F2491FC01BB
:10389000E057FF4F8491882349F190E0880F991FEA
:1038A000FC01E854FF4FA591B49182559F4FFC0154
:1038B000C591D4919FB7611108C0F8948C9120955F
:1038C00082238C93888182230AC0623051F4F89459
:1038D0008C91322F309583238C938881822B88831F
:1038E00004C0F8948C91822B8C939FBFDF91CF9171
:1038F0000895A1E0B0E0EFE7FCE10C944F21282F00
:1039000030E0F901E859FF4F8491F901E458FF4F85
:103910001491F901E057FF4F04910023C9F0882367
:1039200021F069830E94171C6981E02FF0E0EE0FFF
:10393000FF1FE255FF4FA591B4919FB7F8948C916A
:10394000611103C01095812301C0812B8C939FBF0F
:103950002196E4E00C946B21CF93DF93282F30E085
:10396000F901E859FF4F8491F901E458FF4FD491D0
:10397000F901E057FF4FC491CC2391F081110E94CF
:10398000171CEC2FF0E0EE0FFF1FEC55FF4FA59139
:10399000B4912C912D2381E090E021F480E002C0CD
:1039A00080E090E0DF91CF9108958E3008F08E5046
:1039B00087702091B50190E4299F90011124822BFA
:1039C00080937C0080917A00806480937A0080915B
:1039D0007A0086FDFCCF809178002091790090E0FC
:1039E000922B0895A0E0B0E0E8EFFCE10C944B21AD
:1039F0006C017A01EB01E60EF71E00E010E0CE1537
:103A0000DF0561F06991D601ED91FC910190F081A3
:103A1000E02DC6010995080F191FF1CFC801CDB7D8
:103A2000DEB7E8E00C9467216115710589F0DB01D0
:103A30000D900020E9F7AD0141505109461B570B8D
:103A4000DC01ED91FC910280F381E02D0995089550
:103A500080E090E008950E94141D0895DC01ED912E
:103A6000FC910190F081E02D099508950F931F932B
:103A7000CF93DF93EC016DE00E942E1D8C016AE074
:103A8000CE010E942E1D800F911FDF91CF911F91BB
:103A90000F9108950F931F93CF93DF93EC010E9432
:103AA000141D8C01CE010E94361D800F911FDF91E5
:103AB000CF911F910F9108950F931F93CF93DF9391
:103AC000EC010E942E1D8C01CE010E94361D800F3C
:103AD000911FDF91CF911F910F910895A1E2B0E066
:103AE000E4E7FDE10C9447217C01C42EE52FCB01D6
:103AF000D22E19A221E02D1510F02AE0D22E8E012F
:103B00000F5D1F4F8D2C912CA12CB12C6C2D7E2F75
:103B1000A50194010E9400218C2DD29E80191124B0
:103B2000015011098A3010F4805D01C0895CF801F0
:103B30008083211531054105510521F0C22EE32F67
:103B4000CA01E4CFB801C7010E94141DA196ECE0A0
:103B50000C946321A0E0B0E0E0EBFDE10C944B217C
:103B6000EC016A017B012115310541F4E881F981FD
:103B70000190F081E02D642F09951DC02A30310598
:103B8000A9F477FF12C06DE20E942E1D8C0144271C
:103B90005527BA014C195D096E097F092AE0CE014B
:103BA0000E946E1D800F911F06C02AE0B701A6017A
:103BB000CE010E946E1DCDB7DEB7E8E00C94672100
:103BC0000F931F93CF93DF93EC019A01AB0166270C
:103BD00057FD6095762F0E94AA1D8C01CE010E9490
:103BE000361D800F911FDF91CF911F910F91089586
:103BF0002115310549F4DC01ED91FC910190F08132
:103C0000E02D642F099508950E946E1D08959A0174
:103C1000462F50E060E070E00E94F81D08959A0180
:103C2000AB0160E070E00E94F81D0895FC0124855E
:103C30003585F901E05CFF4F80819181F901EE5BF0
:103C4000FF4F20813181821B930B8F739927089539
:103C5000FC0184859585FC01E05CFF4F408151812A
:103C6000FC01EE5BFF4F208131814217530741F089
:103C70000190F081E02DE80FF91F808190E0089518
:103C80008FEF9FEF0895FC0184859585FC01E05C32
:103C9000FF4F40815181FC01EE5BFF4F208131815C
:103CA0004217530779F0A081B181A80FB91F8C91F9
:103CB000208131812F5F3F4F2F7333273183208342
:103CC00090E008958FEF9FEF0895FC0181A1882374
:103CD00029F0A489B5898C9186FFFBCF11A20895A4
:103CE000CF93DF93FC0126853785D901A05CBF4FB8
:103CF0008D919C91119701968F739927E901CE5B65
:103D0000DF4F4881598184179507D9F30D90BC91F5
:103D1000A02DA20FB31F6C93A685B785A05CBF4FE3
:103D200011969C938E93A689B7892C9181E090E09F
:103D3000078C02C0880F991F0A94E2F7282B2C9356
:103D400081E081A30488F589E02D808180648083EF
:103D500081E090E0DF91CF91089508951F920F9236
:103D60000FB60F9211242F933F934F938F939F93EE
:103D7000EF93FF938091C00082FD1CC04091C6006C
:103D80008091BC049091BD0401968F739927209176
:103D9000BE043091BF048217930771F0E091BC0418
:103DA000F091BD04E458FB4F40839093BD04809391
:103DB000BC0402C08091C600FF91EF919F918F914A
:103DC0004F913F912F910F900FBE0F901F9018951C
:103DD00086E194E00E94161E892B11F00E94AD1E10
:103DE00008951F920F920FB60F9211242F933F93B5
:103DF0008F939F93EF93FF932091780430917904F0
:103E000080917A0490917B042817390731F48091CE
:103E1000C1008F7D8093C10014C0E0917A04F091BD
:103E20007B04E85CFB4F208180917A0490917B04B5
:103E300001968F73992790937B0480937A04209343
:103E4000C600FF91EF919F918F913F912F910F901D
:103E50000FBE0F901F901895A0E0B0E0E2E3FFE1E5
:103E60000C944721FC011382128288EE93E0A0E0BB
:103E7000B0E084839583A683B7838AEC92E0918334
:103E800080837587648757874687318B208B138B98
:103E9000028BF58AE48AD78AC68AB18EA08E938E69
:103EA000828E8F85848F8889858F8989868F8A897C
:103EB000878F8B8980A3ECE00C946321CF92DF92F3
:103EC000EF92FF92CF93DF93EC016A017B014115E2
:103ED00081EE580761057105F9F0EC89FD8981E0F3
:103EE00090E008A002C0880F991F0A94E2F780832F
:103EF00060E079E08DE390E0A70196010E94002147
:103F00002150310941095109569547953795279513
:103F1000211580E1380798F0EC89FD89108260E86E
:103F200074E88EE190E0A70196010E9400212150E3
:103F30003109410951095695479537952795E889E3
:103F4000F9893083EA89FB89208319A2EE89FF89E8
:103F5000408181E090E09C010C8C02C0220F331F55
:103F60000A94E2F7422B4083EE89FF8940819C014D
:103F70000D8C02C0220F331F0A94E2F7422B4083BC
:103F8000EE89FF8940819C010E8C02C0220F331FF5
:103F90000A94E2F7422B4083EE89FF8920810F8C3F
:103FA00002C0880F991F0A94E2F7809582238083CC
:103FB000DF91CF91FF90EF90DF90CF900895BF9267
:103FC000CF92DF92EF92FF92CF93DF93EC016A01E1
:103FD0007B01B22E411581EE580761057105F9F09C
:103FE000EC89FD8981E090E008A002C0880F991F4C
:103FF0000A94E2F7808360E079E08DE390E0A70126
:1040000096010E940021215031094109510956951C
:10401000479537952795211580E1380798F0EC8969
:10402000FD89108260E874E88EE190E0A7019601B6
:104030000E940021215031094109510956954795A7
:1040400037952795E889F9893083EA89FB892083A8
:10405000E88DF98DB082EE89FF89408181E090E0A2
:104060009C010C8C02C0220F331F0A94E2F7422BF2
:104070004083EE89FF8940819C010D8C02C0220F94
:10408000331F0A94E2F7422B4083EE89FF89408177
:104090009C010E8C02C0220F331F0A94E2F7422BC0
:1040A0004083EE89FF8920810F8C02C0880F991F01
:1040B0000A94E2F7809582238083DF91CF91FF906D
:1040C000EF90DF90CF90BF9008958F929F92AF9224
:1040D000BF92CF92DF92EF92FF920F931F9381E0F6
:1040E0008F9385E08F9387E08F9383E08F9384E0B5
:1040F0008F93E6EC8E2E912CF2ECAF2EB12CA1EC2E
:10410000CA2ED12CB0ECEB2EF12C04EC10E025ECF7
:1041100030E048E354E06CE774E086E194E00E940C
:104120002C1F0F900F900F900F900F901F910F91D9
:10413000FF90EF90DF90CF90BF90AF909F908F90C7
:1041400008950E94DC1B0E947412C8EEDEE10E94FA
:1041500066162097E1F30E94E81EF9CFA29FB001F6
:10416000B39FC001A39F700D811D1124911DB29FAB
:10417000700D811D1124911D08950E94AE20A59FF0
:10418000900DB49F900DA49F800D911D1124089552
:10419000B7FF0C94BD200E94BD20821B930B089595
:1041A000DB018F939F930E94BD20BF91AF91A29F8F
:1041B000800D911DA39F900DB29F900D1124089525
:1041C000991B79E004C0991F961708F0961B881F69
:1041D0007A95C9F780950895AA1BBB1B51E107C0CA
:1041E000AA1FBB1FA617B70710F0A61BB70B881F87
:1041F000991F5A95A9F780959095BC01CD01089516
:10420000A1E21A2EAA1BBB1BFD010DC0AA1FBB1FDA
:10421000EE1FFF1FA217B307E407F50720F0A21B4C
:10422000B30BE40BF50B661F771F881F991F1A94B9
:1042300069F760957095809590959B01AC01BD01E3
:10424000CF010895052E97FB1EF400940E9439219A
:1042500057FD07D00E94002107FC03D04EF40C94B8
:10426000392150954095309521953F4F4F4F5F4FE5
:10427000089590958095709561957F4F8F4F9F4FD2
:1042800008952F923F924F925F926F927F928F92FA
:104290009F92AF92BF92CF92DF92EF92FF920F93D5
:1042A0001F93CF93DF93CDB7DEB7CA1BDB0B0FB6DF
:1042B000F894DEBF0FBECDBF09942A88398848889C
:1042C0005F846E847D848C849B84AA84B984C88432
:1042D000DF80EE80FD800C811B81AA81B981CE0F29
:1042E000D11D0FB6F894DEBF0FBECDBFED0108950E
:1042F000EE0FFF1F0590F491E02D0994FB01DC0106
:1043000002C001900D9241505040D8F70895F9999C
:10431000FECF92BD81BDF89A992780B50895262FCA
:10432000F999FECF1FBA92BD81BD20BD0FB6F8949A
:0E433000FA9AF99A0FBE01960895F894FFCFFD
:10433E000000C004200008409CFF0088130002000B
:10434E00020002000200020002000200020002004F
:10435E00020002000200020002000200020020051C
:10436E00220623072B0821082709240A250A280AD2
:10437E00290A2A8025000005400AA1204EA500200A
:10438E00244EA52C2330C01200001A400AA1204E44
:10439E00A5001B1E27522C23308025000005400A45
:1043AE00A1204EA50020244EA52C2330004B00004A
:1043BE0006400AD0009D49007B289D492C233000E1
:1043CE00E1000005400A4501D7DC03B81E0EBF0010
:1043DE00232E48E801008A400A6001555502AD1EA1
:1043EE0020000023C80154582074696D656F7574E0
:1043FE00210057616974696E672062696E640A00F4
:10440E00476F7420706B740A006461746120676F6B
:10441E006F640A007363616E6E6572206D6F646502
:10442E00004F70656E4C52536E6720525820737455
:10443E00617274696E672000206F6E2048572000ED
:10444E0053617665642062696E64206461746120D4
:10445E00746F20454550524F4D0A004920616D2022
:10446E00736C61766500456E746572696E67206E59
:10447E006F726D616C206D6F646500454550524FD3
:10448E004D2064617461206E6F742076616C696476
:10449E00206F722062696E64206A756D707065722D
:1044AE00207365742C20666F7263696E6720626973
:1044BE006E640A0052582068616E6700B200F40103
:1044CE004C0300070B0C10111500090E0F101112E2
:1044DE00130A0300010200000001000002000004A4
:1044EE00000008000010000020000400000000087A
:1044FE0000000100000200000000701EF21C161EDB
:06450E00431E281E651E7D
:107E00000F92CDB7DEB7112484B714BE81FFF1D035
:107E100082E08093C00088E18093C10086E0809377
:107E2000C20080E18093C4008EE0CDD088249924E4
:107E3000CC24C394F5E0DF2EE1E1EE2E73E0F72EC3
:107E4000B6D0082F813479F4B2D08983C2D0898129
:107E5000823811F481E005C0813811F485E001C059
:107E600083E09ED09AC0823411F484E103C085344B
:107E700019F485E0B6D091C0853561F498D0082F0B
:107E800010E095D090E0982E8824802A912A880CC2
:107E9000991C82C0863521F484E0A3D080E0E1CF34
:107EA000843609F04CC083D082D0A82E80D0B82E62
:107EB00000E011E07CD0F80181938F01AE16D1F77C
:107EC00088D0FB2DF53489F4E0E0F1E00BC0F9999E
:107ED000FECF92BC81BC0894811C911C819180BD15
:107EE000FA9AF99AEA1598F358C08B2D863409F05E
:107EF00054C0F401F7BEE89507B600FCFDCFF401CD
:107F0000A0E0B1E02C9130E011968C91119790E0B7
:107F1000982F8827822B932B12960C01C7BEE895C9
:107F20001124329681E0A038B80761F7F401D7BE7A
:107F3000E89507B600FCFDCFE7BEE8952EC0843774
:107F4000F1F435D034D0182F32D0B82E42D0FB2DDA
:107F5000F63421F4F40105914F010CC0FB2DF534EA
:107F600049F4F999FECF92BC81BC0894811C911C04
:107F7000F89A00B5802F14D0115049F70EC08537FC
:107F800039F427D08EE10CD085E90AD08FE069CF93
:107F9000813511F488E017D01CD080E101D050CF9A
:107FA0009091C00095FFFCCF8093C600089580910A
:107FB000C00087FFFCCF8091C00084FD01C0A89560
:107FC0008091C6000895E0E6F0E098E19083808318
:107FD0000895EDDF803219F088E0F5DFFFCF84E10E
:107FE000DFCF1F93182FE3DF1150E9F7F2DF1F9166
:0E7FF0000895282E80E0E7DFEE27FF27099492
:027FFE0001057B
:0400000300007E007B
:00000001FF
